:020000020000FC
:020000000CC032
:10001800F7C001E20EBF0FEF0DBF07E104B908E01A
:1000280005B901E00DBD00E50CBD289A2C980F9A82
:1000380017980000179A0CE000936A0000E20DBBC5
:1000480040E8D3D07DD003EC2898C9D001E0C7D0D0
:10005800289A0000000000000000000000000000D6
:100068000000000000000000000000000000000088
:100078005FEFBBD00BEE009364000EE300936500C6
:1000880000E900BF00EE2898AAD006E6A8D0289A72
:1000980001EE2898A4D006E6A2D0289A02EE289865
:1000A8009ED003EC9CD0289A03EE289898D004EAB6
:1000B80096D0289A08EC289892D003E390D0289AF2
:1000C80005EC28988CD000E88AD0289A0CEE28985D
:1000D80086D00EE084D0289A0EEE289880D003E0CF
:1000E8007ED0289A0DEE28987AD000E378D0289A06
:1000F8000FE8289874D0289A0EEC289870D008E059
:100108006ED0289A08E00093C90001E00093CC0063
:10011800B2E0AA27ED010FEF0CBB789451D0000094
:100128000000000000000000AC1709F4F8CF0091AF
:10013800C80005FFFCCF0991D2700093CE00EFCF25
:1001480002EC28984CD008E04AD0289A01E8289870
:1001580046D000E044D0289A0830C1F7089502EC50
:1001680028983DD003E03BD0289A0000000000000A
:10017800000001E8289833D000E031D0289A0830F0
:1001880071F7089502EC28982AD009E028D0289A17
:1001980001E8289824D000E022D0289A0930C1F735
:1001A800089502EC28981BD009E119D0289A01E893
:1001B800289815D000E013D0289A0931C1F708957E
:1001C80002EC28980CD006E10AD0289A01E8289871
:1001D80006D000E004D0289A0631C1F708950EBD74
:1001E8000DB507FFFDCF0EB5089500000000000013
:1001F800000000000000000000004A95B1F70895D3
:100208000F930FB70F930FE82898E9DF289A01E8B2
:100218002898E5DF00E0E3DF289A0F31C1F30131C8
:10022800B1F3063151F402E82898D9DF00E0D7DFAE
:10023800289A007E003338F002C091DFC1DF0F91A9
:100248000FBF0F91189500E22898C9DF00E0C7DFBB
:100258000B5001F1F8F0302F00E0C1DF00E0BFDF04
:1002680000E0BDDFF016A1F000E0B9DF00E0B7DF85
:1002780000E0B5DF00E0B3DF00E0B1DF00E0AFDFB2
:1002880000E0ADDF0D93B2703A95D1F7289AD7CF39
:08029800289AD5CF289AD3CF94
:00000001FF
